:1008FB0000C000F900A400B000990092008200F83B
:10090B00008000900088008300C600A10086008E46
:0A0B7B00E51125E0F511EF4211220B
:0D0AFE00E51125E0F511EFF454014211223D
:040BF300EF5211228A
:070BB000EFF4540152112281
:040BF700EF42112296
:070BB700EFF454014211228A
:0E0AD400E511F45401FFE51154FE4FF5112217
:060BE100E5115401FF22A2
:0D0B0B00E511C313FFE51154015FF5112240
:0D0B1800E511C313FFE51154014FF5112243
:0409C600135401FDC8
:0E09CA00E51125E0F511EDF45F540142112214
:0E0AE200E51125E0F511EFF45D5401421122FB
:08000300EDF45F5401521122DB
:080B9800EFF45D54015211223B
:080BA000EDF45F540142112243
:080BA800EFF45D54014211223B
:070BBE00EDF45F5401FF227A
:070BC500EFF45D5401FF2273
:0D0B2500E51825E0FFE51154014FF51822F9
:0D0B3200E5185401FFE51154FE4FF51122A6
:1009B300E5185401FFE51154FE4FF511E518C31373
:0309C300F5182202
:100AB5008E5D8F5EE55E2DFFE55D3C8FF002049651
:1009D8008E5F8F60C3E5609DFFE55F9C8FF002042A
:0109E8009678
:090B8F001203D5EE8FF00204966A
:0F0AC5008B5A8A5B895C1203E7EE8FF00204966E
:070BCC00E475F00102045E74
:070BD30074FFF5F002045E5F
:1009E9008E618F62E5615CFFE5625DCF8FF0020485
:0109F9009667
:1009FA008E638F64E5634CFFE5644DCF8FF002048C
:010A0A009655
:100A0B008E658F66E5656CFFE5666DCF8FF0020432
:010A1B009644
:100A1C00EFF4FFEEF4FEEF2401FFE43E8FF002044E
:010A2C009633
:060BE700EFF45401FF22AF
:060BED00EE8FF0020496F9
:0A0B8500EFF4FFEEF48FF002049687
:1008A5008B4B8A4C894D120433FFAEF0AB4EAA4FE9
:1008B500A950120433FDAB4BAA4CA94DE5F08DF0C0
:0F08C500120496AB4EAA4FA950EE8FF002049684
:100594008E518F528B538A5489557C037DE8120304
:1005A400E7EFC454F07B00FAAE51AF527C037DE810
:1005B4001203E78C518D52AE51AF527C007D641210
:1005C40003E7EFFEE4EE4202AE51AF527C007D64DD
:1005D4001203E78C518D52AE51AF527C007D0A124A
:1005E40003E7EFC4F8540FC868FFEEC454F048FEA4
:1005F400EFFBEE4202AE51AF527C007D0A1203E7DC
:100604008C518D52E5514AFFE5524BAB53AA54A984
:0706140055CF8FF0020496A0
:10069A008E568F57E557780CCEA2E713CE13D8F8AB
:1006AA007E00540FFF7C037DE81203D58E588F59C4
:1006BA00E556FF3395E07E00EF540FFF7C007D6422
:1006CA001203D5EF2559F559EE3558F558E557AEC9
:1006DA00567804CEA2E713CE13D8F87E00540FFF43
:1006EA007C007D0A1203D5EF2559F559EE3558F5E8
:1006FA0058E557540F2559F559E43558F558855991
:04070A00F00204965F
:10091B00E51125E0F511C3EF9DEC6480F8EE6480E2
:0B092B00984004431101225311FE22EA
:10093600E51125E0F511D3EF9DEC6480F8EE6480B7
:0B094600985004431101225311FE22BF
:10095100E51125E0F511D3EF9DEC6480F8EE64809C
:0B096100984004431101225311FE22B4
:10096C00E51125E0F511C3EF9DEC6480F8EE648091
:0B097C00985004431101225311FE2289
:10098700E51125E0F511EF6D7002EE6C600443117F
:0609970001225311FE22B3
:10099D00E51125E0F511EFB50508EEB50404431199
:0609AD0001225311FE229D
:100A2D00C3EF9DEC6480F8EE64809850035311FE83
:010A3D002296
:100A3E00D3EF9DEC6480F8EE64809840035311FE72
:010A4E002285
:100A4F00D3EF9DEC6480F8EE64809850035311FE51
:010A5F002274
:100A6000C3EF9DEC6480F8EE64809840035311FE60
:010A70002263
:0C0B3F00EFB50507EEB504035311FE22CC
:0C0B4B00EF6D7002EE6C60035311FE228F
:100A7100C3EF9DEC6480F8EE64809840034311015C
:010A81002252
:100A8200D3EF9DEC6480F8EE64809850034311012B
:010A92002241
:100A9300D3EF9DEC6480F8EE64809840034311012A
:010AA3002230
:100AA400C3EF9DEC6480F8EE648098500343110119
:010AB400221F
:0C0B5700EF6D7002EE6C60034311012290
:0C0B6300EFB50507EEB5040343110122B5
:070BDA00E4FF0FBF0AFC223B
:10087500E4FEC2B4120BDAC2B3120BDAD2B3120B16
:10088500DAD2B4120BDAE4FDEE25E0FE3094034330
:100895000601C2B3120BDAD2B30DBD08EBAF0622C7
:1001F4000510E510C394054003E4F510E510146000
:100204005B1470030202B01470030202FC24036046
:100214000302034E7C0090000DE0540FFD25E0FF27
:10022400EC33FE74FB2FF58274083EF583E493FCF3
:10023400740193FD43040890010AE0FFC4131313EF
:10024400540130E0057DFF0203A4EF131313541F80
:1002540020E0030203A453057F0203A490000CE0F2
:10026400FEA3E07804CEA2E713CE13D8F87C0054A2
:100274000FFD25E0FFEC33FE74FB2FF58274083E7E
:10028400F583E493FC740193FD43040490010BE0B3
:1002940030E0057DFF0203A490010AE0FFC4540F7F
:1002A40020E0030203A453057F0203A490000CE0A2
:1002B400FF3395E07C00EF540FFD25E0FFEC33FEA7
:1002C40074FB2FF58274083EF583E493FC74019368
:1002D400FD43040290010BE0FFC31330E0057DFFF2
:1002E4000203A490010AE0FFC413540720E00302B0
:1002F40003A453057F0203A490000CE0FEA3E0785E
:100304000CCEA2E713CE13D8F87C00540FFD25E0E1
:10031400FFEC33FE74FB2FF58274083EF583E493FF
:10032400FC740193FD43040190010BE0FF1313548B
:100334003F30E0047DFF806890010AE0FFC413139E
:10034400540330E05B53057F805690010BE0F9C401
:100354001313540175F008A4FBAAF0E9C413131392
:10036400540175F010A4FFE5F04AFAEF4BFBE9C421
:1003740013540175F004A4FFEA45F0FAEB4FFBE9CE
:10038400C4540125E0FFE4334AFEEB4FFFE91313A5
:10039400135401FBEEEF4BF4FFEEF47410FCAD07C5
:1003A4007B10C2B3120BDAEC20E704C2B78002D28E
:1003B400B7120BDAED25E0FDEC33FCD2B3120BDA05
:1003C400DBE0D2B7120BDAC2B5120BDAD2B5020BEC
:0103D400DA4E
:10000E00E52E70030201F3152E0517E517B405173B
:10001E00AF30EFC4135401F45401FFC43354E0FF66
:10002E00E53054DF4FF530E517B40A1CAF30EFC49E
:10003E00135401F45401FFC43354E0FFE53054DF90
:10004E004FF530051DE4F517E4F568E56813131355
:10005E00541F2412F8E6FD7C00E5685407FF740176
:10006E007E00A807088005C333CE33CED8F9FFEE45
:10007E005CFEEF5D4E6043E56825E025E0246EF5FD
:10008E0082E43400F583E0FEA3E0FFE56825E02579
:10009E00E0246CF582E43400F583E0FCA3E0C39F1A
:1000AE00EC9E5016E56825E025E0246CF582E434DC
:1000BE0000F583E475F00112041DE56825E025E0E6
:1000CE00246EF582E43400F583E0FEA3E0FFE568DC
:1000DE0025E025E0246CF582E43400F583E0FCA3F2
:1000EE00E0C39FEC9E407AE56825E025E0246CF5A0
:1000FE0082E43400FEC3E582946CFFEE9400FE7C35
:10010E00007D021203E77C007D021203E77C007D76
:10011E00081203E7741E2FF8C000E6FFC007E5685B
:10012E0025E025E0246CF582E43400FEC3E58294DC
:10013E006CFFEE9400FE7C007D021203E77C007DD6
:10014E00021203E77C007D081203E7AF057401A8D5
:10015E0007088002C333D8FCFED0E04ED000F680F4
:10016E0079E56825E025E0246CF582E43400FEC3D1
:10017E00E582946CFFEE9400FE7C007D021203E794
:10018E007C007D021203E77C007D081203E7741EDB
:10019E002FF8C000E6FFC007E56825E025E0246CD7
:1001AE00F582E43400FEC3E582946CFFEE9400FE0B
:1001BE007C007D021203E77C007D021203E77C00C7
:1001CE007D081203E7AF057401A807088002C33348
:1001DE00D8FCF4FED0E05ED000F60568E568642039
:0601EE006003020059222B
:1007BB00E51DB41E19AF30EFC413135401F45401EB
:1007CB00FFC4333354C0FFE53054BF4FF530E51D44
:1007DB00B43C1CAF30EFC413135401F45401FFC4E9
:1007EB00333354C0FFE53054BF4FF530E4F51D22D1
:03000B0002070EDB
:10070E00C0E0C0D075D008758CEEAF30EF13131368
:10071E005401F45401FF33333354F8FFE53054F7EA
:10072E004FF530053AE53A30E0020516E53AB40ADF
:10073E0015AF30EFC45401F45401FFC454F0FFE57B
:10074E003054EF4FF530E53AB4141AAF30EFC454CD
:10075E0001F45401FFC454F0FFE53054EF4FF5306F
:0A076E00052E753A00D0D0D0E0321D
:100778007594FF752F05E4F530F53190000CF0A362
:10078800F090010BE054F7F054EFF054DFF054BF51
:10079800F0547FF090010AE054F7F054EFF054DF82
:1007A800F054BFF0547FF0A3E054FEF054FDF05431
:0307B800FBF02231
:040BFB00752F092227
:1007FB00E4FFEF25E025E0246CF582E43400F5837B
:10080B00E4F0A3F00FBF20EAE4FF7F4090002CE45C
:10081B00F0A3DFFCE4FF741E2FF8E4F60FBF04F621
:0D082B00E4FF74192FF8E4F60FBF04F62265
:0E0AF000758911D2B4D2B9D2A9D28CD2AF225C
:10083800AFA0EFC3135455FEEF25E054AA4EFF13A3
:10084800135433FEEF25E025E054CC4EFF54F0FE60
:10085800E590540F4EF4F522EF540FF4540FF5239E
:0D086800120875EFF4F5248528800201F4D4
:10061B00E4FF74222FF8E6FE743F2FF8A6060FBFF7
:10062B0006F0E4FF74282FF8E6FE74452FF8A606B3
:10063B000FBF06F0E4FF74692FF8E6FE74202FF568
:10064B0082E43401F583EEF00FBF20EAE4FF74EC93
:10065B002FF582E43400F583E0FE74402FF582E43D
:10066B003401F583EEF00FBF20E4E4FF741E2FF886
:10067B00E6FE74362FF8A6060FBF04F0E4FF7419DC
:0F068B002FF8E6FE74322FF8A6060FBF04F022F8
:1008D4007567011207781207FB120AF01208381222
:1008E400050A12000E1207BB12061BE56760EDE451
:0708F400F567120BFB80E524
:10050A00AF2FEF13135401FF120B7BE51130E007F5
:10051A00E490010CF0A3F0E5225401FFE53F5401F9
:10052A00FD1209CAE51130E0097B017A01790C1242
:10053A000BCCAF22EFC3135401FFAE3FEEC3120937
:10054A00C6E51130E0097B017A01790C120BD3AFB1
:10055A0022EF13135401FFAE3FEE131209C6E51141
:10056A0030E007E490010CF0A3F0E52F5401FF12EC
:10057A000B7BE51130E01190010CE0FEA3E0FF7B5C
:0A058A00017A00790C120BED00223B
:03000000020B6F81
:0C0B6F00787FE4F6D8FD7581880208D478
:1003D500EF8DF0A4A8F0CF8CF0A428CE8DF0A42E3C
:0203E500FE22F6
:1003E700C2D5EC30E709B2D5E4C39DFDE49CFCEE31
:1003F70030E715B2D5E4C39FFFE49EFE1204B5C3F0
:10040700E49DFDE49CFC80031204B530D507C3E4EA
:060417009FFFE49EFE229F
:10041D00C5F0F8A3E028F0C5F0F8E582158270026A
:06042D001583E038F02207
:10043300BB010A89828A83E0F5F0A3E02250068794
:10044300F009E71922BBFE07E3F5F009E319228956
:0B045300828A83E493F5F07401932289
:10045E00BB010789828A8302041D500B09C5F02750
:10046E00F7C5F01937F722BBFE0D09F8E325F0F3B7
:10047E00C5F019E338F322F889828A837401932533
:08048E00F0C5F0F8E4933822F8
:10049600BB010A89828A83F0E5F0A3F0225006F7B1
:0F04A60009A7F01922BBFE06F3E5F009F31922AE
:1004B500BC000BBE0029EF8DF084FFADF022E4CC2B
:1004C500F875F008EF2FFFEE33FEEC33FCEE9DECF4
:1004D500984005FCEE9DFE0FD5F0E9E4CEFD22ED3A
:1004E500F8F5F0EE8420D21CFEADF075F008EF2F84
:1004F500FFED33FD4007985006D5F0F222C398FD75
:050505000FD5F0EA2211
:00000001FF
